:020000040000FA
:020000009F2D32
:08000800FF000308FE000A08D6
:10001000FC000408FD008312031300308A00233023
:100020008100A10A063021020318A1012014A20FA9
:100030001C28A30F1C28A0143D08003E03193C28CF
:100040002E1C3A2883160313DB3086008312031319
:10005000860106155B230130652300001E30A400D5
:10006000061107306523061506306523A40B3028DA
:1000700006115E285B233E28502349231430A50037
:10008000FB01FA01EF21F521032254238501210808
:1000900003196920013021020319AA20023021022C
:1000A0000319EB200330210203192C210430210213
:1000B00003196D21053021020319AE210B118B1795
:1000C0007D0884007C088A007E088300FF0E7F0E76
:1000D0000900B830840001080002031C7A17B93007
:1000E000840001080002031CFA167A16BA30840054
:1000F00001080002031CFA15BB308400010800024D
:10010000031C7A15A330840001080002031CFB16AF
:10011000A230840001080002031C7B16FB15A130ED
:10012000840001080002031C7B15A0308400010834
:100130000002031CFB14831603137B0885007A0856
:100140008600831203138030860001308500A50BE2
:1001500069280800BC30840001080002031CFA175B
:10016000BD30840001080002031CFA16BE30840072
:1001700001080002031C7A16FA15BF30840001083A
:100180000002031C7A15A730840001080002031C3A
:10019000FB167B16A630840001080002031CFB1529
:1001A000A530840001080002031C7B15A4308400E4
:1001B00001080002031C7B14831603137B088500CF
:1001C0007A088600831203134030860002308500CF
:1001D000A50BAA280800C030840001080002031CF7
:1001E000FA17C130840001080002031C7A17C230DC
:1001F000840001080002031C7A16C3308400010841
:100200000002031CFA157A15FB16AB3084000108B6
:100210000002031C7B16AA30840001080002031CA4
:10022000FB15A930840001080002031CFB14A83050
:10023000840001080002031C7B14831603137B084F
:1002400085007A088600831203132030860004306C
:100250008500A50BEB280800FA17C43084000108BC
:100260000002031C7A17C530840001080002031C39
:10027000FA16C630840001080002031CFA15C730C4
:10028000840001080002031C7A15AF3084000108C5
:100290000002031CFB16AE30840001080002031CA0
:1002A0007B16AD30840001080002031C7B15AC30C6
:1002B000840001080002031CFB147B148316031343
:1002C0007B0885007A0886008312031310308600AD
:1002D00008308500A50B2C290800C83084000108CF
:1002E0000002031CFA177A17C930840001080002C3
:1002F000031CFA16CA30840001080002031C7A1697
:10030000CB30840001080002031C7A15B33084004E
:1003100001080002031CFB16B23084000108000231
:10032000031CFB15B130840001080002031C7B157F
:10033000FB14B030840001080002031C7B148316F8
:1003400003137B0885007A088600831203130830A4
:10035000860010308500A50B6D290800CC30840084
:1003600001080002031CFA17CD30840001080002C6
:10037000031C7A17FA16CE30840001080002031C11
:100380007A16CF30840001080002031CFA15B7303A
:10039000840001080002031C7B16B63084000108AB
:1003A0000002031CFB157B15B53084000108000218
:1003B000031CFB14B430840001080002031C7B14EE
:1003C000831603137B0885007A08860083120313C3
:1003D0000430860020308500A50BAE2908000310EC
:1003E000260DAF00FC21B20008000310260D013ECF
:1003F000AF00FC21B300080002308A002F08073E3E
:1004000003188A0A820032088A0033088200023404
:1004100047340234523402345A34023462340234DF
:100420006A340234723402347A3402348634023448
:100430008A340234963402349A340234A6340234B4
:10044000AA340234B6340234BA340234C634023424
:10045000CA340234D6340234DA340234E634023494
:10046000EA340234F6340234FA3403340634033402
:100470000A340334163403341A3403342634033470
:100480002A340334363403343A34033446342D10DA
:100490003030B10028184F2A0630A600482B013012
:1004A000A600482B2818572A0030A600482B0230F7
:1004B000A600482B28185F2A0030A600482B0330DE
:1004C000A600482B2818672A0430A600482B0330C2
:1004D000A600482B28186F2A0030A600482B0530AC
:1004E000A600482B2818772A0730A600482B003092
:1004F000A600482B2818842A003031070319822AC5
:10050000B10B482B2D14482BA601482B2808AC0012
:10051000A60A482B2C082806031D902AA601482B62
:1005200028182B10281C2B14A60A482B2808AC00CE
:10053000A60A482B2C082806031DA02AA601482B32
:1005400028182A12281C2A16A60A482B2808AC00AC
:10055000A60A482B2C082806031DB02AA601482B02
:100560002818AA11281CAA15A60A482B2808AC008E
:10057000A60A482B2C082806031DC02AA601482BD2
:1005800028182A11281C2A15A60A482B2808AC006E
:10059000A60A482B2C082806031DD02AA601482BA2
:1005A0002818AA10281CAA14A60A482B2808AC0050
:1005B000A60A482B2C082806031DE02AA601482B72
:1005C00028182A10281C2A14A60A482B2808AC0030
:1005D000A60A482B2C082806031DF02AA601482B42
:1005E0002818A912281CA916A60A482B2808AC000E
:1005F000A60A482B2C082806031D002BA601482B11
:1006000028182912281C2916A60A482B2808AC00ED
:10061000A60A482B2C082806031D102BA601482BE0
:100620002818A911281CA915A60A482B2808AC00CF
:10063000A60A482B2C082806031D202BA601482BB0
:1006400028182911281C2915A60A482B2808AC00AF
:10065000A60A482B2C082806031D302BA601482B80
:100660002818A910281CA914A60A482B2808AC0091
:10067000A60A482B2C082806031D402BA601482B50
:1006800028182910281C2914A60A482BA601301462
:1006900008002D10AD10871E2D14871FAD14080003
:1006A0002810071B2814080027082602031C5A2BB1
:1006B0002608A70008002E10BD030310BC0CBB0CBD
:1006C000BA0CB90C03182E140800B400B40B662B36
:1006D0000800BA01BB01BC01A030B900B709371C42
:1006E0003A143718BA14351E3A15351ABA15B51D0D
:1006F0003A16B519BA16351D3A173519BA17B51C79
:100700003B14B518BB14351C3B153518BB15B61E6C
:100710003B16B61ABB16361E3B17361ABB17B61D4C
:100720003C14B619BC14361D3C153619BC15B61C44
:100730003C16B618BC16361C3C173618BC172130B0
:10074000BD000800BE01BF010830C0000310C20C8C
:10075000BF0DBE0DC10CBF0DBE0DC00BA62B0800FA
:10076000C300C4010830C5000310C30CC40DC50B81
:10077000B42B44080800C6000000C60BBC2B0800C0
:10078000CD0A4D080F3C0319CD014D08B800F90101
:10079000F8010800CD034D08013E031DD22B0E3099
:1007A000CD00B800F901F80108002908CD00B80013
:1007B000F13E031CDF2B0E30CD024D08D82BF90182
:1007C000F8010800C7002010201CE42BC70BE32B06
:1007D00008004D0AB023CF00D001D101D201D301CE
:1007E000D40170305718D000FF30EB24CF01D00176
:1007F000D1010130EB2408000530C800EE30C900FB
:1008000003104D0DF9008B13E1258B17CA0003145B
:100810004D0DF9008B13E1258B17C9004A08C8005C
:10082000080021304802031D192C49087907462485
:100830002B2C8B130A08CB0048087807DB00031029
:1008400049087907DC000318DB0AE825CC004B08CF
:100850008A004C088B17F90F2E2CF80A0800831613
:1008600003178C18312C8B130C158312031779087E
:100870008D0077088C008316031755308D00AA3041
:100880008D008C148B178312031308008B138316AF
:1008900003178C18492C0C11831203178D00831633
:1008A00003178C130C14831203170C088312031301
:1008B0008B17080000304624D70008005A24571C24
:1008C000632C5710642C57140030F9005708F700B8
:1008D0002F24E923E9230800FC23F901F80111245E
:1008E000CE00CE131124D600D60A1124D800301C15
:1008F000952C07302A02031D802CD523B0016C2CC7
:10090000AA08031D952C203029020319C023213089
:1009100029020319CA23003029020319CD010C3022
:10092000290203195E24B0016C2C2D080319AB2C8D
:10093000E923E92303302D0203195E242D18A32C8B
:10094000AD18A72C6C2CC023E923E9239A2CCA23C9
:10095000E923E9239A2C17304E0204308A00031948
:10096000D82404308A001B304E0208308A00031954
:10097000002804308A003D08003E031DCB2CA01C3B
:10098000CB2CA010571CC62CC0236C2C0730B500F4
:100990003808B6006923D80B772C6C2C590D590DEB
:1009A000591A013AD91A013AD919013AD90008005D
:1009B0001124CF001124D0001124D1001124D20021
:1009C0001124D3001124D4003030DA005608EB246F
:1009D000DA0BE62C0800D500CC3084008001CF1B58
:1009E0008009C830840080014F1B8009C930840011
:1009F0008001CF1A8009CA30840080014F1A800913
:100A0000CE3084008001CF198009CF30840080016E
:100A10004F198009C13084008001CF188009BC3093
:100A2000840080014F188009C03084008001D01BF1
:100A30008009C43084008001501B8009C5308400C7
:100A40008001D01A8009CD3084008001501A8009BD
:100A5000BB3084008001D0198009BA308400800145
:100A600050198009C33084008001D0188009C63035
:100A70008400800150188009C73084008001D11B98
:100A80008009CB3084008001511B8009BD30840077
:100A90008001D11A8009B83084008001511A800980
:100AA000B93084008001D1198009BE3084008001F2
:100AB00051198009C23084008001D1188009BF30EB
:100AC00084008001511880095508E2230800023093
:100AD0002602031C0301CF000030D0000130EB24BC
:100AE0002D080319832DA701A6013D08003E031D13
:100AF000702D2D08D000CF010130EB24B5010C3052
:100B0000B6006923702D301C672DB001F030CF0086
:100B1000D0017F30EB24CF01D0013F30EB24F03007
:100B2000CF00D0017F30EB242908CF002A08D00065
:100B3000FF30EB24FF30EB24A701A601672D8501D0
:100B40008101CD01BD01AB01AA01A901AC01A60142
:100B5000A701B001A101A201A301AD0183160313F6
:100B600071308F04831603178801890183160313DC
:100B70008230810083160313E03087008312031351
:100B8000AD011D30D9008B168B17FF30CF00D00080
:100B9000D100FF30EB24FF30EB24CF01D001D10195
:100BA000FF30EB24FF30EB24FF30EB245A242D08D8
:100BB000D000FF30EB24FF30EB242D1C6C2C5E2486
:100BC000672D48088A007908490703188A0A8200B5
:100BD0000A08CB005B088A005C0882000834B7343E
:100BE00009344A3409345F340934F2340A340D3498
:100BF0000A34A0340A34B5340A34EE340B340334E6
:100C00000B3418340B343F340B348A340C3429340D
:080C10000D3416340D3461347B
:10100000D50004308A001124CF001124D00011240F
:10101000D1001124D2001124D3001124D4000830AF
:101020008A006430BF00CC308400CF1BAF20CF1FBC
:10103000B320C83084004F1BAF204F1FB320C930EE
:101040008400CF1AAF20CF1EB320CA3084004F1ABD
:10105000AF204F1EB320CE308400CF19AF20CF1D5C
:10106000B320CF3084004F19AF204F1DB320C130C3
:101070008400CF18AF20CF1CB320BC3084004F18A1
:10108000AF204F1CB320C0308400D01BAF20D01F36
:10109000B320C4308400501BAF20501FB320C53094
:1010A0008400D01AAF20D01EB320CD308400501A57
:1010B000AF20501EB320BB308400D019AF20D01D0C
:1010C000B320BA3084005019AF20501DB320C33074
:1010D0008400D018AF20D01CB320C6308400501834
:1010E000AF20501CB320C7308400D11BAF20D11FCC
:1010F000B320CB308400511BAF20511FB320BD3033
:101100008400D11AAF20D11EB320B8308400511A08
:10111000AF20511EB320B9308400D119AF20D11DAA
:10112000B320BE3084005119AF20511DB320C2300E
:101130008400D118AF20D11CB320BF3084005118D7
:10114000AF20511CB320550803308A00E223083039
:101150008A00BF0B1328831304308A00BB2C800A3B
:101160000319800908008008031D80030800173454
:1011700010341834803400340034803400340034A7
:10118000403400340034403400340034203400341F
:10119000003420340034003410340034003410346F
:1011A000003400340834003400340834003400348F
:1011B0000434003400340434003400340234003485
:1011C000003402340034003401340034003401347B
:1011D000003400340034803400340034803400346F
:1011E00000344034003400344034003400342034BF
:1011F000003400342034003400341034003400341F
:10120000103400340034083400340034083400341E
:101210000034043400340034043400340034023424
:10122000003400340234003400340134003400341B
:10123000013400340034003480340034003480340D
:10124000003400344034003400344034003400347E
:10125000203400340034203400340034103400349E
:1012600000341034003400340834003400340834BE
:1012700000340034043400340034043400340034C6
:1012800002340034003402340034003401340034B9
:1012900000340134173410340334FF34FF34FF3486
:1012A000FF34FF34FF34FF34F0340034FF34F034C3
:1012B000003400340F34FF3400340F34FF3417345B
:1012C0000334183480341034003480341034003443
:1012D000403420340034403420340034203440344E
:1012E000003420344034003410348034003410345E
:1012F00080340034093400340034093400340034BC
:1013000006340034003406340034003480341034A1
:1013100000348034103400344034203400344034FD
:10132000203400342034403400342034403400343D
:1013300010348034003410348034003409340034E4
:1013400000340934003400340634003400340634E8
:1013500000340034003408340134003408340134DB
:1013600000340434023400340434023400340234CF
:1013700004340034023404340034013408340034BA
:101380000134083400340034903400340034903494
:1013900000340034603400340034603400340834E5
:1013A000013400340834013400340434023400348D
:1013B000043402340034023404340034023404347B
:1013C000003401340834003401340834003400346B
:1013D00090340034003490340034003460340034ED
:1013E00000346034173410340434FC340F34C03407
:1013F0000034003400341F348134F83400340034B5
:1014000000340334F0343F34003400340034E0342A
:101410007E3407340034003400341B341034183464
:10142000FF34FF34FF34FF34FF34FF34FF34FF3424
:10143000FF34FF34FF34FF34FF34FF34FF34FF3414
:10144000FF34FF34FF34FF34FF34FF34FF34FF3404
:1014500000340034003400340034003400340034EC
:1014600000340034003400340034003400340034DC
:1014700000340034003400340034003400340034CC
:10148000FF34F0340034FF34F0340034FF34F034EF
:101490000034FF34F0340034FF34F0340034FF34CF
:1014A000F0340034FF34F0340034FF34F0340034CE
:1014B000003400340034003400340034003400348C
:1014C000003400340034003400340034003400347C
:1014D000003400340034003400340034003400346C
:1014E00000340F34FF3400340F34FF3400340F3431
:1014F000FF3400340F34FF3400340F34FF34003431
:101500000F34FF3400340F34FF3400340F34FF3411
:10151000003400340034003400340034003400342B
:10152000003400340034003400340034003400341B
:10153000003400340034003400340034003400340B
:10154000173403340334DB346D34B634DB346D3498
:10155000B6346D34B634DB346D34B634DB34B63483
:10156000DB346D34B634DB346D3417340234093473
:101570004F342434F2340034003400344F342434F3
:10158000F2340034003400344F342434F234003464
:10159000003400344F342434F23400340034003446
:1015A0004F342434F2340034003400344F342434C3
:1015B000F2340034003400340F340434F234003494
:1015C000003400344F342434F23400340034003416
:1015D0000F340434F234003400340034173403344C
:1015E0000334DB3460340034DB34603400346D3475
:1015F000B03400346D34B0340034B634D0340034F8
:101600006D34B034003417340334033400340D34F3
:10161000B63400340D34B63400340634DB340034D0
:101620000634DB3400340B346D3400340B346D3449
:10163000173403340634C33401348634C3340134DC
:10164000863461348034C33461348034C3343034FC
:10165000C83461343034C834613418346C343034B4
:1016600018346C3430340C34363418340C3436348A
:101670001834863413340C34863413340C341B344D
:1016800003340C3480347E340134003400340034AC
:10169000C0343C340334003400340034E0341834B3
:1016A0000734003400340034F03400340F34003494
:1016B00000340034783400341E34003400340034F4
:1016C0003C3400343C340034003400341E340034E4
:1016D00078340034003400340F340034F0340034F3
:1016E0000034003407348134E034003400340034F2
:1016F0000334C334C0340034003400340134E734DC
:1017000080340034003400340034FF3400340034BA
:10171000003400341B3403341A3480341034003461
:10172000803410340034C03430340034C0343034A9
:101730000034E03470340034E03470340034F03479
:10174000F0340034F034F03400347934E0340034D0
:101750007934E03400343F34C03400343D34C03494
:1017600000341F34803400341F34803400340F348C
:10177000003400340F3400340034063400340034B4
:1017800006340034003400340034003400340034B3
:1017900000340034003400340034003400340034A9
:1017A0000034003400340034003400340034003499
:1017B0000034003400340034083401340034083478
:1017C000013400340C34033400340C34033400345A
:1017D0000E34073400340E34073400340F340F3421
:1017E00000340F340F34003407349E34003407348F
:1017F0009E3400340334FC3400340334FC340034AD
:101800000134F83400340134F83400340034F03456
:1018100000340034F03400340034603400340034D8
:1018200060340034003400340034003400340034B8
:101830000034003400340034003400340034003408
:1018400000340034003400340034003400340034F8
:1018500000341B3403342734063400340034063497
:10186000003400340F34003400340F3400340034BA
:101870001F34803400341F34803400343F34C0348B
:1018800000343D34C03400347934E03400347934E9
:10189000E0340034F034F0340034F034F034003408
:1018A000E03470340034E03470340034C034303408
:1018B0000034C03430340034803410340034803488
:1018C0001034003400340034003400340034003468
:1018D0000034003400340034003400340034003468
:1018E0000034003400340034003400340034003458
:1018F0000034003400340034603400340034603488
:1019000000340034F03400340034F0340034013456
:10191000F83400340134F83400340334FC34003437
:101920000334FC34003407349E34003407349E34CE
:1019300000340F340F3400340F340F3400340E34BD
:10194000073400340E34073400340C3403340034CC
:101950000C340334003408340134003408340134C6
:1019600000340034003400340034003400340034D7
:1019700000340034003400340034003400340034C7
:1019800000340034003400340034003400340034B7
:101990000634003460340634003460340F340034CC
:1019A000F0340F340034F0341F348134F8341F34F1
:1019B0008134F8343F34C334FC343F34C334FC3412
:1019C0007934E7349E347934E7349E34F034FF348C
:1019D0000F34F034FF340F34E0347E340734E03415
:1019E0007E340734C0343C340334C0343C340334D4
:1019F0008034183401348034183401340034003415
:101A00000034003400340034003400340034003436
:101A10000034003400340034003400340034003426
:101A200000340034003400340034003417340334FC
:101A30000C348034103400348034103400342034BA
:101A4000403400342034403400340934003400344D
:101A500009340034003400340834013400340834CC
:101A600001340034023404340034023404340034C9
:101A70000034903400340034903440342034003446
:101A80004034203400341034803400341034803436
:101A9000003406340034003406340034003400349A
:101AA0000434023400340434023400340134083481
:101AB000003401340834003400346034003400341D
:101AC0006034173401342C34E034003400340034F2
:101AD0000034003400340034003400340034003466
:101AE000E034003400340034003400340034003476
:101AF000003400340034003400340E340034003438
:101B00000034003400340034003400340034003435
:101B100000340E3400340034003400340034003417
:101B20000034003400340034003400340034003415
:101B30000034003400340034003400340034003405
:101B40000034003400340034003400341C340034D9
:101B500000340034003400340034003400340034E5
:101B6000003400341C3400340034003400340034B9
:101B700000340034003400340034003400340134C4
:101B8000C0340034003400340034003400340034F5
:101B90000034003400340134C034003400340034E4
:101BA0000034003400340034003400340034003495
:101BB0000034003400340034003400340034003485
:101BC0000034003400340034003400340034003475
:101BD00003348034003400340034003400340034E2
:101BE00000340034003400340334803400340034D2
:101BF0000034003400340034003400340034003445
:101C000000340034383400340034003400340034FC
:101C100000340034003400340034003438340034EC
:101C20000034003400340034003400340034003414
:101C30000034003400340034003400340034003404
:101C400000340034003400340034003400340034F4
:101C50000034003400347034003400340034003474
:101C60000034003400340034003400340034703464
:101C700000340034003400340034003400340034C4
:101C800000340034003400340734003400340034AD
:101C900000340034003400340034003400340034A4
:101CA000073400340034003400340034003400348D
:101CB0000034003400340034003400340034003484
:101CC0000034003400340034003400340034003474
:081CD00000340034003400343C
:02400E00C428C4
:02401000FF3E71
:02420000FF3489
:00000001FF
